:020000040000FA
:100000008A016E2D000000008716F000030EF1003B
:100010000A08F2000408F300831203138A110A127B
:100020005A298B138B1B11285E30A80060305D2885
:100030008B138B1B18282630A80027305D288B13C4
:100040008B1B1F281330A80014305D288B138B1BCB
:1000500026288930A8000A305D288B138B1B2D2899
:10006000D130A80004305D288B138B1B3428E83076
:10007000A80002305D288B138B1B3B28F430A800AE
:1000800001305D288B138B1B42284930A8000130BA
:100090005D288B138B1B49283130A80001305D2867
:1000A0008B138B1B50282730A80001305D288B1341
:1000B0008B1B57280530A8000130A9002B148B1783
:1000C0002B185F2808008B138B1B6328BC30B600ED
:1000D000BF30A8288B138B1B6A285E30B6006030B7
:1000E000A8288B138B1B71282630B6002730A82830
:1000F0008B138B1B78281330B6001430A8288B1371
:100100008B1B7F288930B6000A30A8288B138B1BE5
:100110008628A130B6000830A8288B138B1B8D28A9
:10012000D130B6000430A8288B138B1B9428E830FC
:10013000B6000230A8288B138B1B9B283130B600E9
:100140000130A8288B138B1BA2280530B600013084
:10015000B700AB148B1708008E018F01C828DF3061
:100160008E00BF30C72800308E00C030C728143042
:100170008E00FE30C728B8308E00FE30C728FA3017
:100180008E00FE30C728DF308E00FF30C7288F007A
:100190008B138B1BC828101463000C1CCC28101068
:1001A0000C108B1708000000000000000000000089
:1001B000000000000000000000000000000000003F
:1001C000000000000000000000000000000000002F
:1001D000000000000000000000000000000000001F
:1001E000000000000000000000000000000000000F
:1001F00000000000000000000000000000000000FF
:1002000001308A0079088207FF34FF34FF34FF345D
:10021000FF34FF34FF34FF34FF34FF34FF34FF3446
:10022000FF34FF34FF34FF347F34FF34FF34FF34B6
:10023000FF34FF34FF34FF34FF34FF34FF34FF3426
:10024000FF34FF34FF34FF347F347F347F34FF3496
:10025000FF34FF34FF34FF34FF34FF34FF34FF3406
:10026000FF34FF34FF34FF347F347F347F347F34F6
:100270007F347F347F347F347F347F347F347F34E6
:100280007F347F347F347F3401308A0079088207DD
:100290000034C034C834D034E034F834FC34FE3494
:1002A000FF34F834FC34FE34FF348034C034E0349E
:1002B000F034F8348B1E4F2D0B1D4F2D0B112B1CC2
:1002C0006629A80B6629A90B66292B10AB1C6D2982
:1002D000B60B6D29B70B6D29AB10BA1990294008E0
:1002E00003198D292A187C292A1483160313F53043
:1002F000D000F830D1008E2983160313D00B8E293D
:10030000D10B8E2983120317A1010030A0008312A4
:1003100003133C14BA133B113C122A10831203132B
:1003200040083D043E043F0442044104031DA72944
:10033000A31BB129C51AB12983120317E80BAF29F2
:10034000E90BAF2983120313A317C516B129A31311
:10035000C51283120317D130E8000430E90083127C
:1003600003130510851083160313880183120313EA
:1003700023088800861386170514CD0A14304D0211
:10038000031DF529CD01FF30880086138617C51C93
:10039000F5292008831384000310840D840D840D37
:1003A000503084070830F80021080004F900840A5E
:1003B0000021013EA40DF80BD42905083C3827057F
:1003C0008500A00A0314A70D04302002031DF129A3
:1003D000A001FB30A700A10A10302102031DF12962
:1003E000A101240888008613861783160313880941
:1003F00083120313851486130808A6000510080845
:10040000A500861783120317351C932A8312031342
:10041000BA1F932A83120317351E242AB60B932A78
:10042000B70B932A3512330820020319392A0730F3
:10043000330203191F2A03303302031D242A351007
:10044000831203133C16372A003020020319932A23
:1004500006303302031D4D2A06302002031D3F2AB9
:100460003516B930B6000630B70083120313C00149
:10047000932A351083120313C001A316932A063062
:100480002002031C492A83120313A3120130C00067
:10049000932A83120313A316462A08303302031D3E
:1004A000562A083020020319392A492A0230330219
:1004B000031D682A02302002031D642A35108312AE
:1004C0000313C001A312932A83120313A312462A13
:1004D00007303302031D7C2A07302002031C492AFF
:1004E00007302002031D432A831203171330B6007E
:1004F0001430B7003516932A03303302031D932AB4
:1005000003302002031C492A03302002031D432A22
:1005100083120313A31A742A831203175A30B600E6
:100520000E30B7007A2A83120317B51C162B8312DC
:1005300003133A1E162B83120317B51EA82AB80BF5
:10054000162BB90B162BB512340828020319BD2A35
:10055000003028020319162B04303402031DD22A5E
:1005600004302802031DC42AB516D130B800043067
:10057000B90083120313BD01162BB5105F1083124F
:100580000313BD012310162B04302802031CCE2AAE
:100590008312031323100530BD00162B831203139F
:1005A0002314CB2A02303402031DDB2A0230280236
:1005B0000319BD2AC82A06303402031DEE2A06306C
:1005C0002802031DE92AB51083120313BD01231469
:1005D000162B06302802031CCE2AC82A0830340203
:1005E000031DF72A083028020319E32ACE2A033014
:1005F0003402031D092B03302802031CCE2A0330CA
:100600002802031DC82A1330B8001430B900B516EB
:10061000162B05303402031D162B05302802031C4F
:10062000CE2A05302802031CC82A032B8312031785
:10063000351D882B83120313BA1E882B83120317D0
:10064000351F312BBC0B882BBD0B882B35133A087B
:1006500010020319442B831203130D30BE008312C2
:10066000031702303A02031D5A2B02301002031DF9
:10067000492B3511402B3517B930BC000630BD0071
:1006800083120313BE01882B351183120313A315A4
:10069000882B023010020318512B83120313A31569
:1006A000542B83120313A3113E08031D882B09301A
:1006B000BE00882B04303A02031D6F2B0430100259
:1006C00003193B2B04301002031C6B2B8312031302
:1006D0000930BE00512B83120313A315542B06308F
:1006E0003A02031D7C2B0630100203193B2B063007
:1006F00010020318512B6B2B08303A02031D882B74
:100700000830100203193B2B08301002031C6B2B1E
:1007100083120317B51DFA2B831203133A1FFA2B0A
:1007200083120317B51FA32BBE0BFA2BBF0BFA2B9B
:10073000B5133B0818020319B62B831203130D30AF
:10074000BF008312031702303B02031DCC2B023083
:100750001802031DBB2BB511B22BB517B930BE0063
:100760000630BF0083120313BF01FA2BB5118312A9
:1007700003132312FA2B023018020318C32B83121F
:1007800003132312C62B8312031323163F08031DE2
:10079000FA2B0930BF00FA2B04303B02031DE12B7A
:1007A000043018020319AD2B04301802031CDD2B92
:1007B000831203130930BF00C32B831203132312C8
:1007C000C62B06303B02031DEE2B06301802031920
:1007D000AD2B063018020318C32BDD2B08303B026B
:1007E000031DFA2B083018020319AD2B083018022C
:1007F000031CDD2B83120317411C042CD40B042C87
:10080000D50B042C41104116C11C0C2CD60B0C2C02
:10081000D70B0C2CC110C116411D142CD80B142C55
:10082000D90B142C41114117C11D1C2CDA0B1C2CA7
:10083000DB0B1C2CC111C117831203138A150A127A
:1008400000288A150A12F5298A150A127D2C8A15A4
:100850000A12632F8A150A12AB2F8A110A16122860
:100860008A150A1606208A150A165B218A110A12B1
:10087000F8013D08031D4707F90044212205031D27
:1008800078143E08031D4807F90044212205031D82
:1008900078173F08031D4907F90044212205031D6D
:1008A000F81778088700F8014008031D4607F9008B
:1008B00044212205031D78154208F9004421220530
:1008C000031D78144108F90044212205031DF81482
:1008D000780889000310A20D031C702C0130A200BF
:1008E000AC0AAD0AAE0AAF0AB40A031D7B2CB00AEB
:1008F000B10AB20AB30A831603134018812CC01838
:10090000B22CC10BB22CC20BB22C9230C100013000
:10091000C20083120313251B952C83160313033087
:10092000430203199E2CC30AA92C8316031300301B
:10093000430203199E2CC303031DA92CC01CA92C20
:100940004010831203138A150A164B238A110A12C8
:10095000B22C430883120313F9008A150A16952551
:100960008A110A1283160313C019B82C401ADA2C04
:10097000C40BDA2CC50BDA2CD130C4000430C5000E
:10098000C60A05304602031DD12CC601401ED12CDB
:10099000C011831203138A150A161B238A110A1227
:1009A000DA2C460883120313F9008A150A16EB2580
:1009B0008A110A1283160313C01AE02C401B032D60
:1009C000C70B3F2DC80B3F2DD130C7000430C800E6
:1009D000C90A05304902031DF92CC901401FF92C31
:1009E000C012831203138A150A1633238A110A12BE
:1009F000DA2C490883120313F9008A150A16F42524
:100A00008A110A123F2D83120313C41B3F2D441B6E
:100A10003F2D83160313C01B1B2D401D3F2D40117E
:100A2000831203138A150A161B238A150A16332309
:100A30008A110A123F2D4015CC0B3F2DCD0B3F2DB7
:100A40001330CC001430CD000130CE064E18342DBA
:100A5000831203133030D500DD00E500ED00D60130
:100A6000DE01E601EE013F2D831203133030D60084
:100A7000DE00E600EE00D501DD01E501ED018312A7
:100A80000313AB1A4F2D83160313CA0B4D2DCB0B3B
:100A90004D2D83120313AB164F2D831203138B18A6
:100AA0008B10831603138C1D5E2D831203138C1D74
:100AB0005E2D8A150A1670238A110A1283120313F7
:100AC0000C1C642D0C10CA0A7308840072088A007A
:100AD000710E8300F00E700E871209002030830023
:100AE000C13081008E018C018D01003085007F3086
:100AF000860018308700FF308800890198017C301B
:100B000092004E3093008312031350308B008C01FF
:100B10008D013C30850086171830870089019801C7
:100B20002430900001309200910136309400203042
:100B300084008001840A80300402031D992DA030B6
:100B400084008001840FA12D831710308400800160
:100B5000840A70300402031DA72D903084008001A8
:100B6000840FAF2D0230C6000330C7000330C80029
:100B7000C9008C1183120313141394138C1DBA2D06
:100B80008C111308141BBA2D831603131419BA2DD4
:100B90008312031372274C3C031DBA2D7227FF00EA
:100BA000163C031DBA2D7227FF077F3C031DBA2D8B
:100BB00072277F07013E031DBA2D7227141BBA2D21
:100BC00083160313141DBA2D831203137F084E3EA0
:100BD000930014168C1DEA2D8C118312031700301C
:100BE000900098000030A0000030A800831203138A
:100BF000A030F4000130A200831603138C154010BE
:100C0000C014C301C0114016C601C0124017C9016B
:100C100083120313FB30A700A00183138A150A1661
:100C200012238A110A12FE30A300FF30A4008101B2
:100C30000B118B168B179B0195019D0197011211CA
:100C400087100711831203175F15DF15831603132F
:100C5000D130CA000430CB00831203130130CE0020
:100C60000330C400C5148A110A16AA228A110A1276
:100C700044083F39031D482E8B138B1B3C2E8A15CD
:100C80000A165D238A110A12BA01BB01BC010D2F9D
:100C90003A18762EBA19762EBA18762E3A19762E7A
:100CA0003B1A762EBB1A762E8B138B1B542E3C1CB4
:100CB000762E3A1A5E2EBB1D3A14762EBA1B632E80
:100CC0003B1DBA15762EBA1A682E3B1CBA14762E26
:100CD0003A1B6D2EBB1C3A15762E3B1B712E3B1614
:100CE000762EBB1B752EBB16762E3C10BC1C0D2F12
:100CF0008B138B1B782E4C1E832E1130C200C1012A
:100D0000C127CD270D2FC201CC1E8B2E1130C10063
:100D1000C127CD270D2FC1014C1F9C2E8A110A1609
:100D2000602792278A110A126E3083120317C200BD
:100D3000C3009427B9270D2FC127CD274C1CB42EF3
:100D40008312031702301002031DAC2E831203130B
:100D5000A3150930BE000D2F8312031300303E028D
:100D6000031DB42EBA140D2FCC1CCA2E83120317E8
:100D700002301802031DC22E8312031323120930FE
:100D8000BF000D2F8312031300303F02031DCA2E34
:100D90003A150D2F4C1DED2EBA1F0D2F8312031780
:100DA00008302002031DDA2E83120313A312013030
:100DB000C0000D2F02302002031DE42E8312031306
:100DC000A3160130C0000D2F831203130030400220
:100DD000031D0D2F0130C0000D2FCC1D0D2F8312D0
:100DE000031706302802031DFB2E83120313231062
:100DF0000530BD000D2F02302802031D052F831280
:100E0000031323140530BD000D2F8312031300308C
:100E10003D02031D0D2F3A140D2F8B17451E122F67
:100E2000F501302FAB1D4B2F3B184D2FBB184D2F0D
:100E30003B194D2FBB194D2FBA184D2F3A194D2F75
:100E4000BA194D2F3A184D2F83120317351B4D2F0A
:100E5000B51B4D2F351A4D2FB51A4D2F8312031385
:100E6000231357207508031D472F8B138B1B352F1A
:100E70003C3085048A150A165D238A110A128B10EC
:100E80000B1663008B100B128B17061C142FAB1163
:100E90002B122317332E2B1A142F83120313AB1E7E
:100EA0005B2F8B138B1B512FAB128A150A160E2248
:100EB0008A110A128B17AB1F6E2F3C186E2F03304E
:100EC0004E02031D6B2F8312031704302802031DEB
:100ED0006C2F83120313AB13831203138A150A16A4
:100EE000FD2D332E8C1D722F8C11130808008312D8
:100EF0000313451C872F1D080319832F451B932FB0
:100F000083120317902F5A309B000C308A2F6B30BE
:100F10009B002C309D009101121583120317C40110
:100F20005F118312031308008312031345187B2FEC
:100F30007A309B002C308A2F83120313451CAC2F70
:100F400017080319A82FC51BB82F83120317B52F35
:100F50005A3095000C30AF2F6B3095002C30970035
:100F60009101121583120317C801DF1183120313B5
:100F70000800831203134518A02F7A3095002C30F7
:100F8000AF2F831203175F15831203134513451800
:100F9000CC2F9B019D018710080083120317DF15DA
:100FA00083120313C5134518D82F95019701071114
:100FB0000800000000000000000000000000000029
:100FC0000000000000000000000000000000000021
:100FD0000000000000000000000000000000000011
:100FE0000000000000000000000000000000000001
:100FF00000000000000000000000000000000000F1
:10100000BA1CD72883120317911C1F28061E12280A
:10101000940195019601920FBE28930A931EBE2853
:101020009110C328940F1528950A01301502031D4D
:10103000BE289110111483120313A311C028111C90
:101040003428061A2C2892019301940FBE28950A81
:10105000951FBE281110C328920A0A301202031DE0
:10106000BE2811109115BE28911D4A28061E402841
:101070009401920FBE28930A931EBE289111C32893
:10108000940A0A301402031DBE289111111595010E
:101090009601BE28111D7228061A56289701940F32
:1010A000BE28950A951FBE281111C328970A0A3039
:1010B0001702031DBE28D42904307802031C6A28B5
:1010C00006307802031CC3281708920093011111FF
:1010D0009115BE2811119116831203130930BE0019
:1010E000A315C028911E8028061E78289401BE28CA
:1010F000940A0A301402031DBE2891121117BE284B
:10110000111F9C28061A86289201BE28920A0A30CE
:101110001202031DBE28111302309000970189307E
:10112000D4000A30D5004114411283120313BA10BF
:10113000BA16BE01A311C028911FB228061EA4280A
:10114000940195019601BE28940FA728950A0930AD
:101150001502031DBE28911391101114831203135D
:10116000A311C02891149201930194019501960155
:1011700083120313A3150930BE00C0288312031382
:101180008A110A12212C1111911783120313A3152E
:10119000C02883120317EC15EC17910190018312FC
:1011A0000313BA103C10BA123B10BE01C028BA1E7D
:1011B0002E293E080319E528831203178930D4002D
:1011C0000A30D50041144112E92883120317411A4D
:1011D000BE2803301002031920290530100203191C
:1011E00020290730100203192029093010020319A1
:1011F000202983120313061A1C2983120317970A46
:1012000014301702031DBE2883120313A3191429D7
:1012100083120317900302301002031925290130AD
:10122000100203192929BE2883120317900A0830D7
:10123000100203182529BE28831203179701BE2820
:1012400083120313061E1C29FD2883120313BE01FB
:10125000C02883120313BA123B14C0283B1CC028B9
:101260003E0803193B29831203178930D4000A3042
:10127000D500411441128312031709301002031DD7
:101280004C290A30900094019501960183120313B2
:10129000A3110D30BE00C0280A301002031D7429AE
:1012A00083120313061A6429831203179701940FFC
:1012B000BE28950A08301502031DBE280B30900089
:1012C00083120313A315492983120317970A1430B5
:1012D0001702031DBE2808309000831203133B1031
:1012E000BA16BE01A315C0280B301002031D8829B1
:1012F00083120313061A8029831203179701BE284D
:1013000083120317970A14301702031DBE286B2996
:1013100001301002031D95290D30900094019501B4
:10132000960183120313A31549290D301002031DE2
:10133000BD2983120313061AAD29831203179701DF
:10134000940FBE28950A07301502031DBE280C30E5
:10135000900083120313A311492983120317970ADC
:101360000A301702031DBE280230900083120313B7
:101370003B10BA16BE01A311C0280C301002031D89
:10138000D32983120313061ACB298312031797015B
:1013900083120313492983120317970A1430170283
:1013A000031DBE28B429BE280310130CF800120C2C
:1013B0009407031CDE29950FDE29960A7808950705
:1013C0000318960AF801120894020318EB29FF305B
:1013D0009507031C960313089502031C9603160D2C
:1013E0000318F429F80AE3295C283A1D092B831213
:1013F0000317991C142A861E072A9C019D019E0131
:101400009A0FB42A9B0A9B1EB42A9910F52A9C0FA6
:101410000A2A9D0A01301D02031DB42A99101914CD
:10142000831203132316B62A191C292A861A212A85
:101430009A019B019C0FB42A9D0A9D1FB42A191082
:10144000F52A9A0A0A301A02031DB42A19109915AE
:10145000B42A991D3F2A861E352A9C019A0FB42A68
:101460009B0A9B1EB42A9911F52A9C0A0A301C0279
:10147000031DB42A991119159D019E01B42A191D45
:10148000672A861A4B2A9F019C0FB42A9D0A9D1F2A
:10149000B42A1911F52A9F0A0A301F02031DB42A23
:1014A0005C2C04307802031C5F2A06307802031C8F
:1014B000F52A1F089A009B0119119915B42A1911D0
:1014C0009916831203130930BF002312B62A991EFE
:1014D000752A861E6D2A9C01B42A9C0A0A301C02B9
:1014E000031DB42A99121917B42A191F922A861AB1
:1014F0007B2A9A01B42A9A0A0A301A02031DB42AD6
:101500001913023098009F018930D6000A30D700A5
:10151000C114C112831203133A11BC123A17BF014E
:101520002316B62A991FA82A861E9A2A9C019D0175
:101530009E01B42A9C0F9D2A9D0A09301D02031D9D
:10154000B42A991399101914831203132316B62A77
:1015500099149A019B019C019D019E018312031322
:1015600023120930BF00B62A831203138312031714
:10157000E51FC12A6513E60BF02AE70BF02AE513F5
:10158000F02A651EE52AE20BC92AE30BC92A651772
:10159000F02AE51EDB2A83120313251AD32A8312AD
:1015A0000317E512F02A83120317E403031DF02A40
:1015B000E5126512F02A83120313251EF22A831204
:1015C0000317E5163230E400F02A83120313251ABC
:1015D000F22A8312031765161330E2001430E30079
:1015E000831203138A110A12242C191199178312DA
:1015F00003132312B62A831203176C16EC179901F2
:101600009801831203133A113C103A13BB10BF0127
:10161000B62A3A1F602B3F080319172B83120317B2
:101620008930D6000A30D700C114C1121B2B831297
:101630000317C11AB42A033018020319522B0530BC
:1016400018020319522B073018020319522B0930C4
:1016500018020319522B83120313861A4E2B83127E
:1016600003179F0A14301F02031DB42A83120313A9
:10167000231E462B83120317980302301802031906
:10168000572B0130180203195B2BB42A831203175E
:10169000980A083018020318572BB42A831203172C
:1016A0009F01B42A83120313861E4E2B2F2B831205
:1016B0000313BF01B62A831203133A13BB14B62ACD
:1016C000BB1C062C3F0803196D2B831203178930AE
:1016D000D6000A30D700C114C11283120317093093
:1016E0001802031D7E2B0A3098009C019D019E016B
:1016F0008312031323160D30BF00B62A0A301802D6
:10170000031DA62B83120313861A962B831203172D
:101710009F019C0FB42A9D0A08301D02031DB42AA4
:101720000B3098008312031323127B2B83120317B1
:101730009F0A14301F02031DB42A08309800831238
:101740000313BB103A17BF012312B62A0B3018023D
:10175000031DBA2B83120313861AB22B83120317AD
:101760009F01B42A831203179F0A14301F02031D1E
:10177000B42A9D2B01301802031DC72B0D30980091
:101780009C019D019E018312031323127B2B0D30BC
:101790001802031DEF2B83120313861ADF2B83120B
:1017A00003179F019C0FB42A9D0A07301D02031DD9
:1017B000B42A0C3098008312031323167B2B831258
:1017C00003179F0A0A301F02031DB42A0230980033
:1017D00083120313BB103A17BF012316B62A0C302D
:1017E0001802031D052C83120313861AFD2B831286
:1017F00003179F01831203137B2B831203179F0A86
:1018000014301F02031DB42AE62BB42ABC1EB62ACC
:1018100083120317191C242C861E112C9C019D0178
:10182000B42A9C0FB42A9D0A05301D02031DB42A58
:101830009D0119109914E5171330E6001430E700E4
:10184000831203132312B62A991C522C861A352CA4
:101850009A019C0F302C9D0A8C301D020318322CEB
:10186000651FB42A831203134E2C9A0A0A301A02F7
:10187000031DB42A0430980083120317BB00B51768
:10188000B930BE000630BF00B5158930D6000A3029
:10189000D700C114C11283120313BC11BC123A1732
:1018A000BF01B62A19149C019D019E0183120313E6
:1018B00023160930BF00B62A03101B0CF8001A0CBF
:1018C0009C07031C662C9D0F662C9E0A78089D07BA
:1018D00003189E0AF8011A089C020318732CFF30A3
:1018E0009D07031C9E031B089D02031C9E031E0DE7
:1018F00003187C2CF80A6B2C512ABA1DAE2D8312CA
:101900000317211CAD2C83120313061F982C83127E
:101910000317A20F8F2CA30AA31E8F2C342FA70A04
:101920000A302702031D9B2CA401A501A601F52E58
:1019300083120317A701A40FF52EA50A0330250271
:10194000031DF52E2110A114E5151330E00014300D
:10195000E10083120313A312F52EA11CCD2C8312D8
:101960000313061BC22C83120317651DBA2C6511C5
:10197000A1103F2DA201A301A40FF52EA50FF52E56
:10198000A110F52E83120317A20A1E302202031D96
:10199000F52EA11021156511F52E211DE82C8312BD
:1019A0000313061FDE2C83120317A401A501A60151
:1019B000A20FF52EA30AA31EF52E342F83120317B0
:1019C000A40A1E302402031DF52E2111A115F52EA7
:1019D000A11D242D83120313061BFE2C8312031753
:1019E000651DF52C6511A1113F2DA701A40FF52E42
:1019F000A50A85302502031CF52EF32C831203174C
:101A0000A70A1E302702031DF52E422F043078024C
:101A1000031C492D0A307802031C142D2708A2004C
:101A2000A301A1112115F52E2708A200A301A111E0
:101A300083120313A31A202D831203172116F52EE8
:101A4000831203172115F52E211E762D8312031301
:101A5000061F352D83120317A401A501A601A20FAD
:101A6000F52EA30AA31EF52E342F83120317A40FFD
:101A7000F52EA50A03302502031DF52E2112A1140F
:101A8000E5151330E0001430E10083120313A316B0
:101A9000F52E83120313A31A582DA31683120317CE
:101AA000E5151330E0001430E100A111A116F52E68
:101AB00083120317A101A201A301A401A501A6019C
:101AC000A7010630A000B3003516B930B6000630C5
:101AD000B70035148930D8000A30D90041154113B8
:101AE00083120313C001BA11BA17F52EA11E8A2D55
:101AF00083120313061F802D83120317A701F52EEF
:101B000083120317A70A1E302702031DF52EA11208
:101B10002117F52E211F9C2D83120313061B942DD4
:101B200083120317A701F52E83120317A70A1E308D
:101B30002702031DF52E582D2114A401A501A6018D
:101B4000A201A301A701E5151330E0001430E10064
:101B500083120313A3160130C000F52EBA1F2B2EDB
:101B600040080319BC2D831203178930D8000A30AE
:101B7000D90041154113C02D83120317411BF52EC7
:101B8000073020020319F22D053020020319F22D2F
:101B9000033020020319F22D83120313061BE62DD6
:101BA00083120317A701A40FF52EA50A0230250200
:101BB000031DF52E83120313A31AE22D83120317BC
:101BC000A0030E2E83120317A00A0E2E83120317F2
:101BD000A70A0A302702031DD32DA701A401A501DE
:101BE000A601F52E83120313061F032E831203177B
:101BF000A701A20A64302202031DF52E83120313EB
:101C0000A31AE22DDE2D83120317A70A0A3027023A
:101C1000031DF92DA701A201A301F52E0930200211
:101C2000031D1A2EA401A501A60183120313BA13E2
:101C30003B15F52E013020020319122E0830200228
:101C4000031D262E83120313C001F52E023020023D
:101C50000319222EF52E3B1DF52E40080319382EB0
:101C6000831203178930D8000A30D9004115411377
:101C70008312031709302002031D5C2E8312031305
:101C8000061B8B2E83120317A40FF52EA50A033013
:101C90002502031DF52EA401A501A601A7010A3006
:101CA000A000E5151330E0001430E10083120313A7
:101CB000A3120130C000F52E01302002031D7C2E3E
:101CC00083120313061BBD2E83120317A40FF52ED8
:101CD000A50A03302502031DF52EA401A501A601C6
:101CE000A7010B30A000E5151330E0001430E1002F
:101CF00083120313A316592E0A302002031DAE2EA1
:101D000083120313061F962E83120317A70A14309B
:101D10002702031DF52E831203170830A000A70128
:101D2000831203133B11BA17C001F52E8312031758
:101D3000A701A40FF52EA50A0A302502031DF52ED2
:101D4000A401A501A6010C30A000E5151330E000A8
:101D50001430E10083120313A316F52E0B3020027A
:101D6000031DE02E83120313061FC82E83120317D0
:101D7000A70A14302702031DF52E83120317023021
:101D8000A000A701831203133B11BA17C001F52E5F
:101D900083120317A701A40FF52EA50A0A30250206
:101DA000031DF52EA401A501A6010D30A000E51527
:101DB0001330E0001430E10083120313A312F52E58
:101DC0000C302002031DEC2E83120313061B842EFD
:101DD00083120317A701F52E0D302002031D342FA7
:101DE00083120313061BB62EE82E83120317E51D7C
:101DF000002F6511E00B2F2FE10B2F2FE5112F2F57
:101E0000651C242FDC0B082FDD0B082F65152F2FE9
:101E1000E51C1A2F83120313A51A122F831203171E
:101E2000E5102F2F83120317DE03031D2F2FE5105C
:101E300065102F2F83120313A51E312F8312031752
:101E4000E5146430DE002F2F83120313A51A312FFF
:101E5000831203176514DC30DC000330DD008312CD
:101E600003138A110A12272C83120317EC16EC179E
:101E7000A101A00183120313BA113C10BA133B1144
:101E8000C001F52E0310230CF800220CA407031C3C
:101E90004C2FA50F4C2FA60A7808A5070318A60AF1
:101EA000F8012208A4020318592FFF30A507031CCC
:101EB000A6032308A502031CA603260D0318622F00
:101EC000F80A512F062D3B1E972F83120317321C41
:101ED000862F83120313261A7B2F83120317B00A4F
:101EE00064303002031D9B2F3210831203133B1208
:101EF0003B17C2019D2F83120317B00183160313F2
:101F0000D40F9B2FD50AD51F9B2FA02F831203130D
:101F1000261E772F831203173214B0018316031382
:101F2000D401D501831203131130C2009D2F3B1F32
:101F30009A2F9D2F9D2F831203138A110A122A2C88
:101F400083120317EC14EC17831203133B123C109B
:101F50003B13C2019D2FBB1EDF2F83120317B21C40
:101F6000CE2F83120313A61AC32F83120317B10AAD
:101F700064303102031DE32FB21083120313BB122E
:101F8000BB17C101E52F83120317B1018316031399
:101F9000D60FE32FD70AD71FE32FE82F831203139F
:101FA000A61EBF2F83120317B214B10183160313A9
:101FB000D601D701831203131130C100E52FBB1FD7
:101FC000E22FE52FE52F831203138A110A122D2C1D
:101FD000831203176C15EC1783120313BB123C100A
:101FE000BB13C101E52F000000000000000000004D
:101FF00000000000000000000000000000000000E1
:102000008A110A12C12F8A110A12CD2F8A110A12BF
:10201000772F8A110A12942F8A110A129C2F8A1183
:102020000A12B92F3A1C272983120317291C3F28AB
:1020300083120313861C2D2883120317AA0F24284A
:10204000AB0AAB1E24287B2AAF0A0A302F02031DDD
:102050003228AC01AD01AE01762A83120317AF011D
:10206000AA01AB01AC0F762AAD0A09302D02031D7F
:10207000762A2910A914831203132310782AA91C85
:102080005E28831203138618542883120317AA01AB
:10209000AB01AC0F4E28AD0F4E28AE0A2E1C762A8F
:1020A0002D1F762AA910952883120317AA0A0A3031
:1020B0002A02031D762AA9102915762A291D7928B6
:1020C00083120313861C6F2883120317AC01AD0122
:1020D000AE01AA0F762AAB0AAB1E762A7B2A8312A0
:1020E0000317AC0A0A302C02031D762A2911A91500
:1020F000762AA91D9B28831203138618832883122E
:102100000317AF01492883120317AF0A0A302F02C1
:10211000031D762A892206307802031C95282F0891
:10212000AA00AB01A911A914762AA91129168312B4
:1021300003132314782A291EB32883120313861845
:10214000AD2883120317AC0F762AAD0A03302D0297
:10215000031D762A2912A916762A83120317AC01C9
:10216000AD01AE01762AA91EC82883120313861C6E
:10217000C32883120317AA0A0A302A02031D762AEB
:10218000A9122917762A83120317AA01AB01762A0E
:10219000291FE328831203138618DA2883120317F2
:1021A000AC0F762AAD0A03302D02031D762A2913BF
:1021B000A917762A83120317AC01AD01AE01AA0F4D
:1021C000762AAB0A762AA91F1A2983120313861CC2
:1021D000112983120317AF0A0A302F02031D762A32
:1021E0008922053078020318FB282F08AA00AB01CA
:1021F000A9132917762AA9010430A800B400B5163E
:10220000D130B8000430B900B5148930DA000A3092
:10221000DB00C115C11383120313BD013A103A1636
:10222000782A83120317AF01AC0F762AAD0F762AF6
:10223000AE0A762A2914AC01AD01AE01AA01AB01A8
:10224000AF018312031323140530BD00782A3A1E10
:10225000072A3D0803193529831203178930DA004C
:102260000A30DB00C115C113392983120317C11BC2
:10227000762A04302802031D582983120313861876
:10228000522983120317AC0F762AAD0A03302D02B0
:10229000031D762A8312031323185029033077294C
:1022A0000530772983120317AC01AD01AE01762A00
:1022B00005302802031D7F2983120313861C7B2906
:1022C00083120317AF0A0A302F02031D762A8312E6
:1022D0000313231C762903304E0203197629053097
:1022E0004E0203197629BD01063077290430831286
:1022F0000317A800762A83120317AF01762A03304A
:102300002802031D9D2983120313861C7B29831237
:102310000317AF0A0A302F02031D762A8312031314
:102320002318762903304E020319762905304E0210
:1023300003197629BD010230772906302802031DD2
:10234000CA29831203138618522983120317AC0F6C
:10235000762AAD0A0A302D02031D762A8312031352
:102360002318B42905307729831203175F1CBA2973
:10237000073077290A30A8008312031323103A127A
:10238000BB150530BD0083120317AC01AD01AE01D2
:10239000AF01762A02302802031DE92983120313B4
:1023A0008618522983120317AC0F762AAD0A0A3019
:1023B0002D02031D762A831203132318E7298312A3
:1023C00003170B30A800831203132314BF29033013
:1023D000772907302802031D012A83120313861C64
:1023E0007B2983120317AF0A0A302F02031D762AB6
:1023F000831203132318FE2906307729BD01083004
:10240000772908302802031D062A762A7B2ABB1D5D
:10241000762A3D080319142A831203178930DA003B
:102420000A30DB00C115C113831203170A302802DA
:10243000031D3B2A83120313861C2B2A83120317C6
:10244000AF0A0A302F02031D762A831203132314C6
:10245000BB113A16732983120317AF01AC0F762A0A
:10246000AD0A05302D02031D762A0C30A800831218
:1024700003132314782A0B302802031D602A8312C9
:102480000313861C502A83120317AF0A0A302F0247
:10249000031D762A831203132310BB113A169A29BF
:1024A00083120317AF01AC0F762AAD0A05302D0257
:1024B000031D762A0D30A800831203132310782AF7
:1024C0000C302802031D6C2A8312031386181E2A5F
:1024D00083120317AF01762A0D302802031D752AD7
:1024E000831203138618432A682A7B2A8312031354
:1024F0008A110A12302C831203176C17EC17A901EA
:10250000A801831203133A103C103A12BB11BD010B
:10251000782A03102B0CF8002A0CAC07031C932A12
:10252000AD0F932AAE0A7808AD070318AE0AF8017A
:102530002A08AC020318A02AFF30AD07031CAE0323
:102540002B08AD02031CAE032E0D0318A92AF80AAE
:10255000982A08008B138B1BAA2A750803193E2F93
:10256000740884008313000D031C322F60300005B3
:10257000031D322F00081F39FC00BE2A12308A00CA
:102580007C088207DF2A822B972BCD2C002D652D0E
:10259000DE2ADE2ADE2ADE2ADE2ADE2ADE2ADE2AFB
:1025A000DE2AB12EB52EB92ED02EF82EFC2E0C2FF1
:1025B000102F202F232F272F2A2F2E2F322F840A40
:1025C000CC3045188005000E00040F39FF00000EC6
:1025D0000005F039FF04BA1E112B7F1C072B7F1A50
:1025E000102B3C19422F001CFF2A831203170830BE
:1025F00010020318052B83120313A3150D2B83124E
:1026000003170330100203180A2B83120313BA1A9C
:10261000BE01112B83120313A3110930BE00112B2D
:10262000D1243A1F372BFF1C2D2BFF1A362BBC1938
:102630004C2F801C252B8312031708301802031817
:102640002B2B831203132312332B83120317033014
:1026500018020318302B831203133A1BBF01372BC8
:102660008312031323160930BF00372BDD24BA1F52
:102670005D2B7F1D532B7F1B5C2B3C1A562F001D9F
:102680004B2B83120317083020020319512B83129E
:102690000313A316592B8312031702302002031DC4
:1026A000562B83120313BA1BC0015D2B8312031335
:1026B000A3120130C0005D2BE9243A1E812BFF1DBF
:1026C000772BFF1B802B801D6F2B83120317063087
:1026D00028020319752B8312031323147D2B8312F5
:1026E000031702302802031D7A2B831203133A1AB0
:1026F000BD01812B8312031323100530BD00812BF4
:10270000F524322F840AFC3045188005FC30000582
:10271000031D322F001C8F2B1130C200902BC201E1
:10272000801C952B1130C100962BC101322F840AD9
:10273000000E0739FC009C2B13308A007C088207AE
:10274000A82BC82BF72B362C722C792C802C322FEF
:102750003C1A562FBA1F3E2F83120317351A3E2FED
:102760008312031307300005FC00BC2383120317F8
:10277000B30035143512322F13308A007C088207DB
:10278000063408340234073403340634063406347D
:1027900083120317B51A3E2F831203133A1E3E2FDE
:1027A000163000020319DF2B07300005FC00EB2375
:1027B00083120317B400B5145F14B512322F8312BD
:1027C0000317A9010030A800A914831203133C14B5
:1027D0003A12BB11322F13308A007C08820704346E
:1027E00006340234083405340334043404343C1908
:1027F000422FBA1E3E2F83120317351B3E2F831222
:102800000313243000020319172C2530000203198A
:10281000182C2630000203191A2C03300005FC0086
:10282000BE012E2483120317BA003515322F322F22
:102830003C15322F831203179101920193019401E9
:102840009501960100309000111483120313A31117
:102850000930BE003C14BA123B10322F14308A00EB
:102860007C0882070234043406340834BC194C2F27
:102870003A1F3E2F83120317B51B3E2F83120313FB
:10288000343000020319562C353000020319572C3E
:102890003630000203195E2C03300005FC00BF0136
:1028A0002E2483120317BB00B515322F322FBC150F
:1028B0003A13BC16831203179901322F83120317A0
:1028C00099019A019B019C019D019E010030980095
:1028D00019148312031323160930BF003C143A1352
:1028E000BB10322F01300005031D322F3B163B1366
:1028F000322F01300005031D322FBB16BB13322FC0
:102900003C19422FBC194C2FBA1E3E2F3A1F3E2FA6
:1029100083120317351B3E2FB51B3E2F8312031363
:10292000643000020319A92C653000020319AA2C97
:10293000663000020319AB2C03300005FC00BE0119
:10294000BF012E2483120317BA00BB003515B5153D
:10295000322F322F322F83120317910199019201E6
:1029600093019401950196019A019B019C019D019F
:102970009E01003090009800111419148312031363
:10298000A31123160930BE00BF003C14BA143A1537
:10299000BA123A133B10BB10322F8A150A16932C29
:1029A000322F83120317910100309000831203131A
:1029B0003C14BA123B103C11080083120317990112
:1029C00000309800831203133C143A13BB10BC115F
:1029D000080083120317A1010030A0008312031323
:1029E0003C14BA133B113C12080083120317A901CF
:1029F0000030A800831203133C143A12BB110800E4
:102A0000840A000803193F2D001C132D001A102DF5
:102A1000BA18132D83120317023010020319112D57
:102A2000D12483120313801C222D801A1F2D3A19E2
:102A3000222D83120317023018020319202DDD24E2
:102A400083120313001D312D001B2E2DBA19312DB9
:102A5000831203170630200203192F2DE924831255
:102A60000313801D3E2D801B3D2D3A183E2D8312F1
:102A700003170430280203193E2DF524642D3C145D
:102A80004518552DBA103A11BA123A133C11BC111F
:102A90003B10BB103B13BB13831203179101990129
:102AA000003090009800831203133A10BA113A12C2
:102AB000BA133C12BB113B1183120317A101A901E8
:102AC0000030A8000030A000322FC301840A000E9D
:102AD0000F39FC0008307C020318A82E831203175C
:102AE0000630B300351483120313441AA82E0330A2
:102AF00080050310800D800D000DFC077F2D153023
:102B00008A0083120317DF107C088207A62DC72DC9
:102B1000EC2D0C2E272E482E632E832EAA2DCD2D84
:102B2000F02D0F2E2B2E4B2E672E892EB72DDA2D42
:102B3000FC2D182E382E542E732E962EBB2DE02DE4
:102B4000002E1B2E3C2E572E772E9C2E60277F2783
:102B5000B430BE2D60277F276E3083120317C2006A
:102B6000C300DF140920B9278A110A16C62D602771
:102B70007F27C830BE2D60277F278C308312031734
:102B8000C200C30006209C278A110A16322F602734
:102B900003208A110A16B430E52D60277F27B43050
:102BA00083120317C3006E30C2000C2094278A11D1
:102BB0000A16EB2D602703208A110A16C830E52D6E
:102BC000602703208A110A168C3083120317C20073
:102BD00006208A110A16322F60279227B430032E5E
:102BE000602792276E3083120317C200C3000920AA
:102BF000B9278A110A160B2E60279227C830032E98
:102C0000602792278C3083120317C200C30006206E
:102C10009C278A110A16322F7327B4301D2E732772
:102C20006E3083120317C20009208A110A16232E60
:102C30007327C8301D2E73278C3083120317C200F0
:102C400006208A110A1603208A110A16322F7327CA
:102C50009227B4303F2E732792276E3083120317CA
:102C6000C200C300DF140920B9278A110A16472EB3
:102C700073279227C8303F2E732792278C308312F8
:102C80000317C200C30006209C278A110A16322FA0
:102C90009227B430592E92276E3083120317C30047
:102CA0000F208A110A165F2E9227C830592E9227BC
:102CB0008C3083120317C3000C208A110A160020DF
:102CC0008A110A16322F73277F27B4307A2E732782
:102CD0007F276E3083120317C200C3000920B92773
:102CE0008A110A16822E73277F27C8307A2E7327FF
:102CF0007F278C3083120317C200C30006209C2755
:102D00008A110A16322F7F2700208A110A16B43042
:102D1000A12E7F276027B43083120317C2006E30C4
:102D2000C3000620B9278A110A16A72E7F27002084
:102D30008A110A16C830A12E7F2700208A110A1690
:102D40008C3083120317C3000C208A110A16322F0D
:102D50008312031300208A110A1603208A110A160F
:102D6000322F8A150A16052D322F840A0008C40056
:102D7000322F83160313840A000801390319C82E61
:102D80004014C0100130C1000130C200C301C92E7F
:102D9000C014000E01390319322F10308007D32ED2
:102DA00083160313840A000E03390319E92E000861
:102DB00001390319E42EC01640130130C700013059
:102DC000C8000430C900E52E4017000E023903196F
:102DD000322F000801390319F62EC01540120130B8
:102DE000C4000130C5000430C600322F4016322F17
:102DF0008A150A168E2A322F840A00080319092F11
:102E0000013000020319062F4516322F2B16AB1185
:102E1000322FAB152B12322F8A150A16D72C322FD0
:102E2000840A000803191C2F83160313C0171330DC
:102E3000CC001430CD00322F83160313C013322F71
:102E40008A150A160D2D8A150A16112D322F4515D1
:102E5000C511322F8A150A161C2D322F8A150A1613
:102E6000322D322F83120313F40AF40AC030740295
:102E7000031C3C2FA030F400F503F5038312031369
:102E80008B1708003C113C14BA123B108312031735
:102E90009101003090003E2FBC113C143A13BB103E
:102EA000831203179901003098003E2F3C123C1406
:102EB000BA133B1183120317A1010030A0003E2F6B
:102EC00083120313A318722F451C702F1D080319BA
:102ED000702F4517831203175F1583120313722F88
:102EE000A3144513080083120313A31C7E2F451C53
:102EF0007C2F1D08031D692FA310451308008312A2
:102F00000313231D912F451C8F2F170803198F2F93
:102F1000C51783120317DF1583120313912F231193
:102F2000C51308008312031323199D2F451C9B2FE3
:102F30001708031D882F2315C51308000000000083
:102F40000000000000000000000000000000000081
:102F50000000000000000000000000000000000071
:102F60000000000000000000000000000000000061
:102F70000000000000000000000000000000000051
:102F80000000000000000000000000000000000041
:102F90000000000000000000000000000000000031
:102FA0000000000000000000000000000000000021
:102FB0000000000000000000000000000000000011
:102FC0000000000000000000000000000000000001
:102FD00000000000000000000000000000000000F1
:102FE00000000000000000000000000000000000E1
:102FF00000000000000000000000000000000000D1
:103000008A110A12C12F8A110A12CD2F83120317B7
:103010005F197528C40A031D1528831203137D3018
:103020001B02031815289B0A37288312031740191F
:10303000272883120313061D342883120317CC0A92
:103040000A304C02031D3728401598283728831270
:1030500003130619342883120317CC0A0A304C02D2
:10306000031D37284011372883120317CC01831220
:10307000031303304E02031D742883120317401EEE
:103080006728CE0B4B28CF0B4B2883120313431713
:103090008A150A16EB29401F5D2883120313A51811
:1030A0005528831203174013722883120317D20383
:1030B000031D722840134012722883120313A51CAB
:1030C00074288312031740173230D20072288312FB
:1030D0000313A51874288312031740161330CE006B
:1030E0001430CF00831203130800EA0AEA1E97285F
:1030F000EA01831203135A301B0203188C28451F60
:1031000088280230A3064513831203175F119728FE
:103110009B019D01871097281D0E0339FF3E031C5C
:103120009428F0309D07972830309D049B03372862
:103130004708F800F7014608C700F8070318F70A20
:103140004508C600F8070318F70A4408C500F80741
:103150000318F70A0310F70CF80C0310F70C780C9F
:1031600042020319DE28031CCD28831203131B0817
:10317000031DC1281D0E0339031DC1289D018710A1
:10318000DE281D0E0339FF3E031CC928F0309D07C1
:10319000DE2830309D049B03DE28831203137D302C
:1031A0001B020318DE281D0E013E03390319DB281C
:1031B00010309D07DE280C309D059B0A83120317F3
:1031C000C40126284B08F800F7014A08CB00F8078D
:1031D0000318F70A4908CA00F8070318F70A48084D
:1031E000C900F8070318F70A0310F70CF80C0310CE
:1031F000F70C780C430203192829031C17298312A2
:1032000003131508031D0B29170E0339031D0B2982
:10321000970107112829170E0339FF3E031C1329B4
:10322000F030970728293030970495032829831216
:1032300003137D30150203185029170E013E033980
:10324000031925291030970728290C309705950A6E
:1032500083120317C801831203131D081707031DE8
:10326000332912114D2983120317DF1C4F298312B2
:1032700003137D301B02031850297C301B020318F6
:103280004D297C30150203184D2983120317C20300
:103290000319C20AC3030319C30A831203177B2944
:1032A00083120317DF1C4F29C20A0319C203C30A82
:1032B0000319C3034F2983120317DF19C829C80A4A
:1032C000031D6A29831203137D30150203186A292E
:1032D000950A8C2983120317C0197C2983120313C2
:1032E000861D892983120317CD0A0A304D02031D5A
:1032F0008C29C015E2288C29831203138619892989
:1033000083120317CD0A0A304D02031D8C29C01108
:103310008C2983120317CD018312031303304E024D
:10332000031DC72983120317C01EBA29D00B9E297B
:10333000D10B9E2983120313C317EB29C01FB02999
:10334000831203132519A82983120317C013C52953
:1033500083120317D303031DC529C013C012C52947
:1033600083120313251DC72983120317C017323098
:10337000D300C529831203132519C7298312031704
:10338000C0161330D0001430D1008312031308008C
:10339000EB0AEB1EEA29EB01831203135A301502E4
:1033A0000318DF29C51FDB290430A306C5138312C8
:1033B0000317DF11EA29950197010711EA29170E72
:1033C0000339FF3E031CE729F0309707EA29303024
:1033D000970495038C298312031740124013C012DF
:1033E000C01383120313A318FB298A110A1660273E
:1033F0008A150A16002A8A110A1673278A150A16D0
:10340000231D082A8A110A167F278A150A16C7293A
:103410008A110A1692278A150A16C729C41A172A6A
:1034200083160313D130CA000430CB001D2A831643
:1034300003134230CA001030CB0083120313C41FA1
:103440003F2A0A304E02031D292A4B08013C003056
:10345000031D3030DF00D7000A304E02031D342A2E
:103460004B08023C3030031D0030D500DD00E50084
:10347000ED00D600DE00E600EE0000304C2A441FCE
:103480005B2A0030DF00D700D500DD00E500ED004D
:10349000D600DE00E600EE00D100D900E100E90030
:1034A000D200DA00E200EA00D300DB00E300EB0028
:1034B000D400DC00E40044080339FC00441E6A2AFE
:1034C0002B1B692A0030D000D800E000E8002B1741
:1034D0008D2A2B131A308A007C088207872A802ABB
:1034E000792A722A3030D000D800E0000030E8009D
:1034F0008D2A3030D800E0000030D000E8008D2A5E
:103500003030E0000030D000D800E8008D2A3030A4
:10351000E8000030D000D800E0000800840A4E081F
:10352000B90000020319FD2A0008CE00063C031969
:1035300045100A304E0203190C2B0C304E020319B1
:10354000062B02304E0203190C2B4B231B23332373
:10355000C413441309304E020319092BAB1707306B
:103560004E020319002BBA1ABE013A1BBF01C20159
:10357000C10100208A150A1603208A150A16033095
:103580004E020319D72A05304E020319EA2A0630E3
:103590004E020319EA2A01304E02031DF32A0230BB
:1035A00039020319FD2A0A3039020319FD2A451888
:1035B000E62ABA123B103A13BB108312031791018B
:1035C00099010030900098008312031301304E02DD
:1035D0000319F32A3A12BB1183120317A901003011
:1035E000A800831203133C14BA133B118312031770
:1035F000A1010030A000831203138A110A16FB2ECA
:103600008A110A16F5248A150A16FD2A8A110A1645
:103610000C2F8A110A160C2FC201C10180018A11D8
:103620000A16E02A4B231B2333230030E800E00076
:10363000D800D00008000A304E02031D232B4B088F
:10364000013C0030031D3030DF000A304E02031D04
:103650002D2B4B08023C003003193030D500DD0023
:10366000E500ED0008000A304E02031D3B2B4B081D
:10367000013C0030031D3030D7000A304E02031DDC
:10368000452B4B08023C003003193030D600DE00D9
:10369000E600EE0008003030D100E200EA00D3007E
:1036A000DB00E300EB00D400DC00E4000030D900D4
:1036B000E100E900D200DA000800071387130911BE
:1036C000071009108910BE01BF01C001BD01C20170
:1036D000C10100208A150A1603208A150A1608005F
:1036E0001308F800141B852C8C118316031314196E
:1036F0008D2C941A7E2B83120313882C83120313B0
:103700004F1C892B4C307802031D852C4F10CF1491
:10371000842CCF18A62B4F1D942B4F11CF15780852
:1037200083160313D300822CCF1D852CCF11831653
:1037300003135208530783120313F7007807013E5F
:10374000031D852C77084E3EB800682CF81FAF2B60
:10375000CF104F15780883160313D200822CD03077
:103760007805031D842C203078050319842C0F3034
:103770007805F900BB2B1B308A0079088207842C5E
:10378000CF2BDA2BE22BEA2BF02B842CF42BF62B0D
:10379000362C3A2C3E2C402C422C442C462CBA1B66
:1037A000D32B0030D82B8312031720088312031366
:1037B000B800842C3A1ADE2B0030D82B8312031762
:1037C0002808D62BBA1AE62B0030D82B8312031701
:1037D0001008D62B3A1FE42B831203171808D62B98
:1037E000B801AB1BB80A842C4308D82B83120317EB
:1037F000EC1FFF2B6C0883120313B800352C8312C7
:103800000313260870390838B8000F302605031D49
:10381000B80A451C352C3C19202C831203170430A0
:103820001002031D1E2C83120313BA1E202C3E0807
:10383000031D202C0230061A202CB8048312031317
:10384000BC19352C8312031704301802031D332CC6
:10385000831203133A1F352C3F08031D352C043007
:10386000861A352CB80483120313842C2608803959
:10387000B800842CB801C519B80A842C4608D82B86
:103880004708D82B4808D82B4908D82BB8013D0841
:10389000031DB8174008031D38173F08031DB8164D
:1038A0003E08031D38164108031DB8154208031DC4
:1038B00038151708031DB8141D08031D381483128A
:1038C0000317FF30410683120313F039B804842C28
:1038D000203075020319842C750874078400C030E9
:1038E0000402031C752CE030840783138316031332
:1038F00052088000840A5308800083120313F50ADB
:10390000F50A842C8312031308001413941314165D
:103910004F14CF104F11CF11842C8312031338088A
:1039200093001416842C840A00080319B72C451838
:10393000D42C3C19422FBC194C2FBA1E3E2F3A1FD3
:103940003E2F83120317351B3E2FB51B3E2F8312CC
:103950000313BE01BF01831203170630BA000430FF
:10396000BB003515B515831203134514D42C451C23
:10397000D42CBA18C62C8312031791010030900082
:10398000831203133C14BA123B103C113A19D32C86
:1039900083120317990100309800831203133C141B
:1039A0003A13BB10BC1145108A110A16D02CC00165
:1039B000BD01BA113A103C10BA133A124518EA2C5C
:1039C000C201C101BE01BF01BA103A11BA123A13C5
:1039D0003B10BB103B11BB1100208A150A160320B7
:1039E0008A150A16831203173512B5123510B51051
:1039F000831203134518022D831203173513B513D1
:103A00003511B5118A110A160F2F840A00087F3963
:103A1000CC00BC148A110A16B42E840A0008CB000C
:103A2000172D840AC51000080319192DC5141B236E
:103A300033238A110A16262F840A000E0339FC004C
:103A400000080339FF002A2584007F0880008A11BE
:103A50000A162D2F1D308A007C0882074634473411
:103A6000483449344514BA103A11BA163A173C1181
:103A7000BC113B10BB103B17BB17BE01BF01C201FD
:103A8000C101831203179101990104309800063097
:103A900090004116C1168A110A16312F3030D3001A
:103AA000DB00E3000030D100D900E100E900D200E2
:103AB000DA00E200EA00EB00D400DC00E4000800D9
:103AC0003030E900EA00D300DB00E300EB00DC006B
:103AD0000030D100D900E100D200DA00E200D400C9
:103AE000E40008003030E100E900D200EA00D30031
:103AF000DB00E300EB00D400DC00E4000030D10088
:103B0000D900DA00E20008003030D100D900E1002D
:103B1000E900D200DA00E200EA00D300DB00E300B3
:103B2000EB00D400DC00E40008001D308A007908B6
:103B300082074E2D602D722D842D3030DF00003035
:103B4000D500DD00E500ED0008003030DF00D500D5
:103B50000030DD00E500ED0008003030DF00D5006A
:103B6000E5000030DD00ED0008003030DF00D5005A
:103B7000E500DD00ED0008003030D500E500DD0097
:103B8000ED000030DF0008003030D7000030D600F4
:103B9000DE00E600EE0008003030D700D60000302E
:103BA000DE00E600EE0008003030D700D600E60068
:103BB0000030DE00EE0008003030D700D600E6000E
:103BC000DE00EE0008003030D600E600DE00EE0039
:103BD0000030D70008001D308A00790882079D2D2B
:103BE000A52DAD2DB52DBC2D1D308A00790882077D
:103BF000C42DCC2DD42DDC2DE32D451D8B2E033073
:103C0000C600C700C800C90010140C100C14A3167D
:103C10000130C000CA018312031708302002031DBF
:103C20000D2E831203134A08FF00C0010330C600A3
:103C300064307F020318272EC60350307F0203181A
:103C4000272EC6033C307F020318272EC6032314F9
:103C50000530BD00CA018312031706302802031D78
:103C60002D2E831203134A08FF00BD010330C70045
:103C700032307F020318472EC70328307F02031813
:103C8000472EC7031E307F020318472EC703A31514
:103C90000930BE00CA018312031706301002031D4B
:103CA0004D2E831203134A08FF00BE010330C800E3
:103CB00041307F020318672EC80337307F02031894
:103CC000672EC8032D307F020318672EC803231206
:103CD0000930BF00CA018312031706301802031D02
:103CE0006D2E831203134A08FF00BF010330C90081
:103CF00041307F020318872EC90337307F02031833
:103D0000872EC9032D307F020318872EC903451162
:103D100010100C100C108A110A12712F00008E2E38
:103D20000000000000000000000000000000000093
:103D30000000000000000000000000000000000083
:103D40000000000000000000000000000000000073
:103D50000000000000000000000000000000000063
:08400000803F883F813F833FB0
:02400E00F23F7F
:00000001FF
